:0C000000830100308A0004288301C22B19
:1006F4008312A101C83083128523A10A0530210287
:10070400031808007C2B8312A2000430A30053308A
:10071400A400A40B8B2BA30B892BA20B872B080003
:100724008312A100A2019B2B0D30A300A30B982BD5
:10073400A20A2108220203180800962B8312A100A2
:10074400A201AA2B0D308312A300A30BA72BA20A8C
:10075400FF30A700A8012108A702031CA803220850
:10076400A500A6012608803AA9002808803A290293
:10077400031DBE2B27082502031CA42B831208008B
:100784008316850107308312990083169F01831213
:10079400850105158510051083127A23051185142A
:1007A40005107A230511851005147A23051585147F
:1007B40005107A230515851005147A23051185146F
:1007C40005147A230515851405147A238501A001DF
:1007D400A00A05152008922305112008A023A00AC9
:1007E400200FEB2BFF30A0000515200892230511E4
:0A07F4002008A023A00BF62B042818
:02400E00C43FAD
:00000001FF
